:100000000C942A000C9447000C9447000C94470071
:100010000C9447000C9447000C9447000C94470044
:100020000C9447000C9447000C9447000C94470034
:100030000C9447000C9447000C9447000C94470024
:100040000C9447000C9447000C9447000C94470014
:100050000C94470011241FBECFE5D8E0DEBFCDBF12
:1000600010E0A0E6B0E0EEE0F3E002C005900D92F3
:10007000A03AB107D9F710E0A0EAB0E001C01D92A4
:10008000A83BB107E1F70E9449000C9485010C944C
:1000900000002F923F924F925F926F927F928F92C9
:1000A0009F92AF92BF92CF92DF92EF92FF920F9307
:1000B0001F93DF93CF93CDB7DEB7C854D0400FB6B0
:1000C000F894DEBF0FBECDBFDE01D396ECE8F0E0C2
:1000D00084E101900D928150E1F78FE387BB8FEFB0
:1000E00084BB81BB18BA8CEF8ABB81E087B986E8F4
:1000F00086B9C598C498FFE16F2E712C6C0E7D1ED9
:10010000F301CE0189961192E817F907E1F7BE01D4
:10011000645E7F4F29967FAF6EAF29971E010894CA
:10012000211C311CE3E38E2E912C8C0E9D1E70EA57
:10013000472E7FE0572EC59A80E28A95F1F7C59841
:1001400080E18A95F1F7FE017596C49885EB8A9552
:10015000F1F7369A3699FECF84B190E025B1B22EF0
:10016000AA248A299B2966E670E00E947101693001
:1001700008F068E06193C49A29968EAD9FAD2997E7
:10018000E817F90711F78D8989A78E898AA78F89C2
:100190008BA7888D8CA7498D242F30E0F901E80FBB
:1001A000F11DCF01959587958DA74EA74A8D842F78
:1001B00090E0280F391F359527952FA748AB2B8D39
:1001C000820F911D9595879589AB2AAB29E2E22E86
:1001D000F12CEC0EFD1EBE01655F7F4FA101D30126
:1001E00000E010E0F70120819C91291728F4FA0122
:1001F0008081981B9C930BC0222341F02F5F2C938E
:100200002150FA011082FB01108201C01C928C91D6
:100210008A3010F0F9E0FC93FB0180818F5F8083CE
:100220008F3030F0FA0180818F5F8083FB01108274
:10023000E22FF0E0EE0FFF1FE05AFF4F20813181E7
:10024000ED91F0E0EE0FFF1FEA58FF4F80819181A2
:1002500082239323F801EC55FF4F9183808382BB67
:1002600026B336E0969587953A95E1F730E0237FFF
:100270003070822B932B88BBF401E00FF11F80813B
:10028000218185BB86B390E08C7F9070C22EDD24E7
:100290008C299D2988BBC2010197F1F70894E11CC4
:1002A000F11C0E5F1F4F6F5F7F4F4F5F5F4FE81472
:1002B000F90409F097CF3FCF8FE387BB8FEF84BB63
:1002C00081BB18BA8CEF8ABB089589E08EBD80E9A6
:1002D00091E09BBD8ABD089581E087B986E886B923
:1002E0000895AA1BBB1B51E107C0AA1FBB1FA6177D
:1002F000B70710F0A61BB70B881F991F5A95A9F7CF
:0E03000080959095BC01CD010895F894FFCF33
:10030E00FF03FE03FC03F803F003E003C0038003C6
:10031E00000300020000FE03FD03FB03F703EF03DF
:10032E00DF03BF037F03FF02FF01FF0380004000D6
:10033E00200010000800040002000100000200016D
:00000001FF
